:100000005328A0002108220403194E284820A401E7
:10001000A501200984178005841300000F282308F8
:10002000A40700082004031C20068000A50A031969
:10003000A10A0319A20F0D282008841780044E2856
:100040008001840AFF3E031D20284E28A401A3003E
:10005000FF30A307031CA407031C4E280330A20093
:10006000DF3034202828A201E83EA100A209FC309C
:10007000031C3D28A10703183A28A1070000A20F7E
:100080003A2821184328A11C4728000047280800C7
:10009000A109A209A10A0319A20A08008313831265
:1000A00003130000080007309900CC308316850048
:1000B0008113831285012030840040302020932852
:1000C000831685128312851285100430A700B03084
:1000D000A6000A302620051971280430A700B03088
:1000E000A600A603260A0319A70327082604031D52
:1000F00069284B30A8000330A700E730A60085141C
:10010000080083160512831205123230262064304F
:10011000A3000730A2000830A10005308400203081
:10012000012060200800051D9628932805148516D7
:1001300085140330A400203027206430A300013050
:10014000A200F430A100053084002030012060209E
:100150002808A300A2010230A1000530840010305D
:1001600001200519B42881202708013A4D300319D0
:100170002606031DBD283F30A800A603260A031942
:10018000A70327082604031DA82883160512831237
:0C01900005128510051093286300CC2890
:02400E00C43FAD
:00000001FF
